:020000040000FA
:04000000E4EF00F039
:0400080080EF0CF089
:080018009AEF0CF00F0B426E91
:10002000000EF76E3A0EF66E4250F626D8B0F72A5A
:10003000F29E0800F28EF550120030313233343522
:1000400036373839414243444546A5D8A7D84F6E84
:10005000F5EC0CF0A3D84F5CF8E1640E4D6E9ED821
:1000600002E2C8EF00F0F5EC0CF04D2EF8D70A0EC6
:100070004F26F0EC0DF0000EF86E1E0EF76E140E0B
:10008000F66E03EC0EF051B832D00B0E4F6208D072
:10009000000EF86E1C0EF76E6C0EF66E03EC0EF092
:1000A0000C0E4F6218D0000EF86E1E0EF76E5C0E2E
:1000B000F66E03EC0EF0000EF86E1E0EF76E680E74
:1000C000F66E03EC0EF0000EF86E1E0EF76E740E58
:1000D000F66E03EC0EF00D0E4F6208D0000EF86EB7
:1000E0001E0EF76E5C0EF66E03EC0EF051D0060E8F
:1000F0006B631CD00B0E4F6209D0000EF86E1D0E04
:10010000F76E9C0EF66E03EC0EF042D00C0E4F62B2
:1001100001D003D00D0E4F6209D0000EF86E1D0EF7
:10012000F76E780EF66E03EC0EF032D0090E6B63AC
:100130002FD00B0E4F620BD051BC2AD0000EF86EA0
:100140001E0EF76EFA0EF66E03EC0EF021D00C0EBA
:100150004F6201D003D00D0E4F621AD051AC18D0AF
:10016000000EF86E1F0EF76E060EF66E03EC0EF024
:10017000000EF86E1F0EF76E120EF66E03EC0EF008
:10018000000EF86E1F0EF76E1E0EF66E03EC0EF0EC
:1001900005D8FEE2120002D8FEE31200E86A50B071
:1001A00007D081A8010E81AA020E81AC030E06D0F1
:1001B00081A8030E81AA020E81AC010EE86602D06E
:1001C000D8901200D8801200A5EC0CF030EC0CF0A6
:1001D0001EEC0CF045EC0DF054EC0CF050A407D0E4
:1001E00078EC0CF02FEC0BF0C1EC0BF002D066ECCD
:1001F0000CF042EC0CF00CEC0CF086EC0DF04E8E9A
:10020000200E6A6FC80E566E518AC0EC09F0CEEC13
:1002100000F07EE325EC00F0010E4F6206D0412A8B
:10022000040E416202D0416A72D0020E4F621DD0AC
:10023000416605D050A4582A50B46F2B3FD0010E10
:10024000416208D050A403D00A0E6F2702D00A0ED4
:10025000582634D0020E416202D0572A2FD0030E06
:10026000416203D00A0E572629D0030E4F623ED0BA
:10027000416605D050A4580650B46F071FD0010E38
:10028000416208D050A403D00A0E6F5F02D00A0E5C
:10029000585E14D0020E416202D057060FD0030EF2
:1002A000416203D00A0E575E09D058AE07D07F0EC8
:1002B000586E04D058BE02D0810E586E50A40DD096
:1002C0006FAF02D06F6B416A320E6F6502D0320E93
:1002D0006F6F2FEC0BF0C1EC0BF05268518257BEE0
:1002E000576A460E576402D0460E576E0B0E4F6289
:1002F00004D0F0EC0DF03CEC04F00C0E4F6202D098
:1003000013EC03F00D0E4F6202D05BEC03F04F6A6A
:100310004E4E4E8E010E4E620AD024EC04F0020EB8
:100320006C6103D014EC0EF002D0BCEC0DF0020EA8
:100330004E6202D00CEC04F0030E4E6202D0D3ECFD
:1003400003F0040E4E620FD051A20DD052660BD0B6
:10035000519250B403D05CEC0CF003D0416A6EECC7
:100360000CF04AEC0CF0050E4E6200D0060E4E6208
:1003700036D04BC12CF04CC12DF04DC12EF04EC1EA
:100380002FF04FC130F084C131F085C132F086C109
:1003900033F087C134F088C135F07AEC17F011E3FF
:1003A00051BA1DD04BC184F14CC185F14DC186F1CC
:1003B0004EC187F14FC188F1300E546E750E556EE7
:1003C0000ED055660CD054660AD04BC184F14CC196
:1003D00085F14DC186F14EC187F14FC188F1070EFD
:1003E0004E6206D051A604D008EC02F0B0EC1BF02F
:1003F000080E4E6205D051AA03D0566601D0519A1C
:10040000090E4E6200D00A0E4E6200D005EF01F0D8
:1004100060C017F061C018F062C019F04AEC12F029
:10042000D6EC13F07AC131F07BC132F07CC133F0ED
:100430007DC134F07EC135F0ECEC13F07FC131F0BA
:1004400080C132F081C133F082C134F083C135F014
:10045000AFEC14F02CC04BF12DC04CF12EC04DF17F
:100460002FC04EF130C04FF157C017F057EC12F0CB
:10047000D6EC13F04BC131F04CC132F04DC133F02A
:100480004EC134F04FC135F0AFEC14F02CC04BF13D
:100490002DC04CF12EC04DF12FC04EF130C04FF1A8
:1004A00058C017F03AEC12F0D6EC13F0BBEC16F093
:1004B0004BC131F04CC132F04DC133F04EC134F07C
:1004C0004FC135F0AFEC14F02CC04BF12DC04CF106
:1004D0002EC04DF12FC04EF130C04FF1120050A28E
:1004E000C5EF1DF0A2EF1DF0000EF86E1F0EF76EA7
:1004F0002A0EF66E06EC0EF025EC1CF0F5EF1DF062
:10050000000EF86E1F0EF76E2E0EF66E06EC0EF055
:10051000EAEC0FF060C017F061C018F062C019F08B
:100520003EEC1AF0376A050E366E1DEC19F012001B
:10053000410E51B22A0ED7EC0DF0EAEC0FF057C085
:1005400017F03EEC1AF0376A020E366E1DEC19F009
:100550001200020E496E58C017F03AEC12F0D6ECB9
:1005600013F0420E356EC60E346E316A326A336A4B
:100570007AEC17F002E3030E496E420E356EC60E9A
:10058000346E316A326A336A357E4AEC17F002E320
:10059000030E496E020E496203D0200ED7EC0DF017
:1005A000BBEC16F056EC1AF0010E376E49C036F06F
:1005B000F8EC19F0398449EC19F0000EF86E1F0EB2
:1005C000F76EB00EF66E06EC0EF012001EEC16F092
:1005D000358E31C084F132C085F133C086F134C02C
:1005E00087F135C088F1546A556AC80E566E518A33
:1005F000120050C043F050940CEC04F043C050F093
:100600001200000EF86E1E0EF76EA40EF66E03ECCE
:100610000EF0EAEC0FF06EC017F03EEC1AF0010E8F
:10062000366E1DEF19F0DBEC0BF0C7EC03F0000E9B
:10063000F86E1E0EF76EB00EF66E03EC0EF0000EA6
:10064000F86E1E0EF76EBC0EF66E03EC0EF0D9DFE0
:1006500025EC00F0020E4F6203D0CDEC03F0E7D79B
:10066000030E4F6203D0C7EC03F0E1D7010E4F62D7
:100670001CD0FBEC0BF089C14BF18AC14CF18BC152
:100680004DF18CC14EF18DC14FF1F0EC0DF0B0EC9D
:100690001BF0D3EC03F0F9EC02F0000EF86E1E0E26
:1006A000F76E980EF66E03EC0EF025EC00F04F6A34
:1006B000F0EC0DF0120084C14BF185C14CF186C104
:1006C0004DF187C14EF188C14FF1B0EC1BF0D3EC76
:1006D00003F0F9EC02F0000EF86E1E0EF76E500EED
:1006E000F66E03EC0EF025EC00F0000EF86E1E0E18
:1006F000F76E5C0EF66E03EC0EF0000EF86E1E0E3A
:10070000F76E800EF66E03EC0EF0000EF86E1E0E05
:10071000F76E500EF66E03EC0EF025EC00F0020EB4
:100720004F6202D053DF30D0030E4F622DD0000E47
:10073000F86E1E0EF76E8C0EF66E03EC0EF0000EC9
:10074000F86E1E0EF76E980EF66E03EC0EF025ECAA
:1007500000F0020E4F6218D0DBEC0BF052DFE7EC3A
:100760000CF084C189F185C18AF186C18BF187C102
:100770008CF188C18DF1F2EC0BF00FD8D1EC0BF0BD
:10078000E7EC0CF0E6EC02F0F0EC0DF012006E0776
:100790006EAF02D0090E6E6F12006E2B0A0E6E63E2
:1007A00001D06E6B1200BCEC0DF0000EF2EC0DF0FF
:1007B0006C6702D06FEF02F0010E6C6302D074EF31
:1007C00002F0020E6C6302D06FEF02F01200200EF6
:1007D000F2EC0DF0EAEC0FF070C017F071C018F0F9
:1007E0003EEC1AF0040E366E1DEC19F0000EF86E99
:1007F0001F0EF76E340EF66E06EC0EF0280EF2ECBD
:100800000DF0EAEC0FF06FC017F03EEC1AF03A84EE
:10081000020E366E1DEF19F050A402D0D8DF13D0AF
:10082000BCEC0DF0200EF2EC0DF06C6702D074EF12
:1008300002F0010E6C6302D06FEF02F0020E6C63E7
:1008400002D074EF02F01200BCEC0DF0400EF2EC9E
:100850000DF06C6704D098EC02F0A9EF02F0010EE5
:100860006C6304D098EC02F0A9EF02F0020E6C6306
:1008700002D080EF02F01200F1EC0CF04F6A5AEC5B
:1008800004F025EC00F0010E4F6201D0BED0020E44
:100890004F6206D06B2B0C0E6B6301D06B6BEED7E7
:1008A000030E4F6206D06B076BAF02D00B0E6B6F5F
:1008B000E5D712006B6709D0000EF86E1C0EF76EBC
:1008C000780EF66E03EC0EF08FD0010E6B6309D03C
:1008D000000EF86E1C0EF76E840EF66E03EC0EF032
:1008E00083D0020E6B6309D0000EF86E1C0EF76EFB
:1008F000900EF66E03EC0EF077D0030E6B6309D00A
:10090000000EF86E1C0EF76E9C0EF66E03EC0EF0E9
:100910006BD0040E6B6309D0000EF86E1C0EF76EE0
:10092000A80EF66E03EC0EF05FD0050E6B6309D0D7
:10093000000EF86E1C0EF76EB40EF66E03EC0EF0A1
:1009400053D0060E6B6309D0000EF86E1C0EF76EC6
:10095000C00EF66E03EC0EF047D0070E6B6309D0A5
:10096000000EF86E1C0EF76ECC0EF66E03EC0EF059
:100970003BD0080E6B6314D050A409D0000EF86E63
:100980001C0EF76ED80EF66E03EC0EF02DD0000E96
:10099000F86E1C0EF76EE40EF66E03EC0EF024D02B
:1009A000090E6B6309D0000EF86E1C0EF76EF00E88
:1009B000F66E03EC0EF018D00A0E6B6309D0000E31
:1009C000F86E1C0EF76EFC0EF66E03EC0EF00CD0FB
:1009D0000B0E6B6309D0000EF86E1D0EF76E080E3D
:1009E000F66E03EC0EF000D0000EF86E1D0EF76EE2
:1009F000140EF66E03EC0EF0000EF86E1D0EF76E80
:100A0000380EF66E03EC0EF0120051886B6701D0C1
:100A100046D0010E6B6302D06C6B3FD0020E6B634D
:100A200003D0010E6C6F39D0030E6B6303D0020E3E
:100A30006C6F33D0040E6B6303D008EC08F02FD03A
:100A4000050E6B6303D057EC05F029D0060E6B63DF
:100A500003D094EC06F023D0070E6B6303D006ECB2
:100A600006F01DD0080E6B6303D059EC05F017D0CB
:100A7000090E6B6303D079EC05F011D00A0E6B639D
:100A800003D047EC06F00BD00B0E6B6306D0507012
:100A900014EC0CF0E7EC0CF0FF0038EC0CF0F0EC90
:100AA0000DF051984F6A416AF1EC0CF01200B0EF72
:100AB00009F0507438EC06F050A407D078EC0CF034
:100AC0002FEC0BF0C1EC0BF002D066EC0CF0120036
:100AD000000EF86E1E0EF76EEC0EF66E03EC0EF0C6
:100AE000A9EF02F002EE00F06FC0E9FFEFCF58F07F
:100AF00012006CC044F06C6B50C043F05094200E58
:100B00006A6FC1EC0BF04F6AF0EC0DF02FEC0BF0BC
:100B1000E7EC03F068EC05F051BC0CD05084BCEC61
:100B20000DF0000EF86E1E0EF76EF20EF66E03EC70
:100B30000EF009D0000EF86E1E0EF76EF60EF66E71
:100B400003EC0EF05094C0EC09F008EC02F0200E1B
:100B50006A6305D0D3EC03F0416A14EC0EF0CEECDE
:100B600000F0F1E325EC00F00B0E4F6203D051AC26
:100B700043D007D00C0E4F6207D051AC02D045C015
:100B800058F0E7EC0CF0BFD70D0E4F6207D051AC18
:100B900002D045C058F0E7EC0CF0B5D7010E4F621B
:100BA00011D051AC0ED0C8EC0BF0000EF86E1E0E3A
:100BB000F76E2C0EF66E03EC0EF058C045F0E7EC25
:100BC0000CF0517C020E4F6205D051AC6F2B51BC22
:100BD000582A07D0030E4F6204D051AC6F0751BCA6
:100BE00058066FAF01D06F6B320E6F6502D0320EB8
:100BF0006F6F51AC86D787D743C050F044C06CF0BC
:100C0000F0EC0DF04F6AE7EC0CF01200F0EC0DF098
:100C1000BCEC0DF0000EF86E1E0EF76EC80EF66EF0
:100C200003EC0EF0000EF86E1E0EF76ED40EF66E8C
:100C300003EC0EF0000EF86E1E0EF76EE00EF66E70
:100C400003EC0EF025EC00F0010E4F6201D0DED770
:100C5000020E4F6202D050920BD0030E4F6202D0B0
:100C6000508206D0030E4F6402D098EF09F00CD0EA
:100C700014EC0CF0F0EC0DF0000EF86E1D0EF76E9B
:100C80009C0EF66E03EC0EF0E7EC0CF01200F0ECAC
:100C90000DF0BCEC0DF0000EF86E1D0EF76ED40ECC
:100CA000F66E03EC0EF0000EF86E1D0EF76EE00E01
:100CB000F66E03EC0EF0000EF86E1D0EF76ECC0E05
:100CC000F66E03EC0EF0EAEC0FF040C017F03EECCD
:100CD0001AF0020E366E1DEC19F025EC00F0020E33
:100CE0004F6202D0402A04D0030E4F620ED040065D
:100CF0003F0E406402D03F0E406E0F0E406002D0A7
:100D00000F0E406EC3EC0DF0D6D7010E4F6204D02B
:100D100026EC0CF03AEF06F0030E4F6404D0F0EC32
:100D20000DF098EF09F01200F0EC0DF0000EF86EE7
:100D30001E0EF76E140EF66E03EC0EF0000EF86E3B
:100D40001E0EF76E200EF66E03EC0EF0E5EC0CF0C6
:100D5000F0EC0DF0000EF86E1E0EF76E2C0EF66E17
:100D600003EC0EF0000EF86E1E0EF76E380EF66EE7
:100D700003EC0EF0000EF86E1E0EF76E440EF66ECB
:100D800003EC0EF0E5EC0CF082EC0AF0416AF0ECBA
:100D90000DF0000EF86E1D0EF76EF80EF66E03ECF9
:100DA0000EF0CFEC0AF0BBEC07F025EC00F0010EE2
:100DB0004F6206D0412A0A0E416201D0416AF1D742
:100DC000020E4F6203D0A5EC07F0EBD7030E4F6283
:100DD00003D0AAEC07F0E5D70B0E4F623FD066C1F7
:100DE00017F067C118F050EC12F027C066F128C068
:100DF00067F129C068F12AC069F12BC06AF16BC1A3
:100E000017F06CC118F050EC12F027C06BF128C03D
:100E10006CF129C06DF12AC06EF12BC06FF1176A19
:100E2000186A196A1A6A1B6A17C070F118C071F142
:100E300019C072F11AC073F11BC074F11E0E176E47
:100E4000176C3AEC12F027C075F128C076F129C072
:100E500077F12AC078F12BC079F1DCD10C0E4F620A
:100E600001D066D20D0E4F6201D062D21200DCECCE
:100E70000FF0416607D066C117F067C118F0010E88
:100E80001C6E62D0010E416207D066C117F067C1C7
:100E900018F00A0E1C6E58D0020E416207D066C1CF
:100EA00017F067C118F0640E1C6E4ED0030E41623D
:100EB00009D066C117F067C118F0E80E1C6E030E6A
:100EC0001D6E42D0040E416209D066C117F067C1A1
:100ED00018F0100E1C6E270E1D6E36D0050E4162E6
:100EE00007D06BC117F06CC118F0010E1C6E2CD02E
:100EF000060E416207D06BC117F06CC118F00A0EE4
:100F00001C6E22D0070E416207D06BC117F06CC176
:100F100018F0640E1C6E18D0080E416209D06BC127
:100F200017F06CC118F0E80E1C6E030E1D6E0CD08D
:100F3000090E416209D06BC117F06CC118F0100E98
:100F40001C6E270E1D6E00D0120037EC07F06FEC00
:100F500013F004D037EC07F05AEC13F0050E4160A3
:100F600005D017C066F118C067F104D017C06BF147
:100F700018C06CF11200B5EC0DF0416602D0290EDC
:100F80002DD0010E416202D0280E28D0020E4162FF
:100F900002D0270E23D0030E416202D0260E1ED0AF
:100FA000040E416202D0250E19D0050E416202D016
:100FB000490E14D0060E416202D0480E0FD0070E23
:100FC000416202D0470E0AD0080E416202D0460E9E
:100FD00005D0090E416202D0450E00D0F2EC0DF0B2
:100FE00012006DC017F03AEC12F0D6EC13F056EC8C
:100FF0001AF0376A020E366E398449EC19F0000E89
:10100000F86E1F0EF76EAC0EF66E06EC0EF01200C8
:10101000F0EC0DF0F60E6D6FBCEC0DF0000EF86EFE
:101020001D0EF76E600EF66E03EC0EF0000EF86EFD
:101030001D0EF76E6C0EF66E03EC0EF0000EF86EE1
:101040001D0EF76E440EF66E03EC0EF0F1EC07F099
:1010500025EC00F0010E4F6201D00AD0020E4F6263
:1010600002D06D2BEBD7030E4F6202D06D07E6D78F
:10107000030E4F6401D05CD16DC017F03AEC12F052
:1010800027C070F128C071F129C072F12AC073F134
:101090002BC074F1200E6A6FF0EC0DF0000EF86EAC
:1010A0001D0EF76E200EF66E03EC0EF0000EF86EBD
:1010B0001D0EF76E2C0EF66E03EC0EF0C0EC09F070
:1010C00022EC0AF0CEEC00F0F9E325EC00F0010E82
:1010D0004F6201D00CD0020E4F6201D008D0030E37
:1010E0004F6201D025D1030E4F6401D021D160C0E1
:1010F00017F061C018F062C019F04AEC12F027C076
:1011000066F128C067F129C068F12AC069F12BC0D7
:101110006AF1F0EC0DF0E20E6D6FBCEC0DF0000E1C
:10112000F86E1D0EF76E600EF66E03EC0EF0000EFC
:10113000F86E1D0EF76E6C0EF66E03EC0EF0000EE0
:10114000F86E1D0EF76E520EF66E03EC0EF0F1EC1B
:1011500007F025EC00F0010E4F6201D00ED0020E18
:101160004F6202D06D2BEBD7030E4F6202D06D079A
:10117000E6D7030E4F6401D0DBD06DC017F03AEC18
:1011800012F027C075F128C076F129C077F12AC086
:1011900078F12BC079F1200E6A6FF0EC0DF0000EA3
:1011A000F86E1D0EF76E200EF66E03EC0EF0000EBC
:1011B000F86E1D0EF76E2C0EF66E03EC0EF0C0EC02
:1011C00009F02EEC0AF0CEEC00F0F9E325EC00F08B
:1011D000010E4F6201D00CD0020E4F6201D008D038
:1011E000030E4F6201D0A4D0030E4F6401D0A0D0F3
:1011F00060C017F061C018F062C019F04AEC12F03C
:1012000027C06BF128C06CF129C06DF12AC06EF1C6
:101210002BC06FF166C12CF067C12DF068C12EF0B4
:1012200069C12FF06AC130F06BC131F06CC132F08E
:101230006DC133F06EC134F06FC135F0A9EC14F01C
:101240002CC00EF12DC00FF12EC010F12FC011F1E6
:1012500030C012F170C12CF071C12DF072C12EF0AE
:1012600073C12FF074C130F075C131F076C132F026
:1012700077C133F078C134F079C135F0A9EC14F0BE
:101280000EC131F00FC132F010C133F011C134F092
:1012900012C135F06CEC14F02CC07AF12DC07BF14A
:1012A0002EC07CF12FC07DF130C07EF166C131F0DF
:1012B00067C132F068C133F069C134F06AC135F0FA
:1012C000ECEC13F0307E70C131F071C132F072C1BC
:1012D00033F073C134F074C135F0AFEC14F02CC0AE
:1012E0007FF12DC080F12EC081F12FC082F130C07E
:1012F00083F1000EF86E1D0EF76E9C0EF66E03EC79
:101300000EF0E7EC0CF002EC0CF03AEC0AF0E5EC35
:101310000CF05FEC0AF0E5EC0CF0F8EC0AF0E5EC10
:101320000CF082EC0AF0C5EC0AF0E5EC0CF00AD007
:10133000000EF86E1D0EF76E780EF66E03EC0EF0D2
:10134000E7EC0CF04F6A1200E5EC0CF0000EF86EC2
:101350001D0EF76E900EF66E03EC0EF025EF00F00A
:101360003AEC0AF0F1DF5FEC0AF0EEDFF8EC0AF09D
:10137000EBDF82EC0AF0C5EC0AF0E6DF4F6A120000
:101380003BEC0DF0196A59C017F05AC018F017500D
:101390005D2618505E2219505F226A2F52D0200E0F
:1013A0006A6FD890653766376737D8906537663784
:1013B0006737DCEC0FF05DC017F05EC018F05FC05F
:1013C00019F0175065271850662319506723EAEC67
:1013D0000FF065C017F066C018F067C019F0050E71
:1013E0001C6E52EC18F017C065F018C066F019C0FA
:1013F00067F0020E1C6405D0652BD8B4662BD8B4F8
:10140000672B6751625D05E16651615D02E16551DF
:10141000605D0000D8B009D0640E536E65C060F006
:1014200066C061F067C062F008D0536606D065C040
:1014300060F066C061F067C062F05D6A5E6A5F6A14
:1014400051861200BCEC0DF0000EF86E1D0EF76E0A
:101450004A0EF66E03EC0EF088EF02F0BCEC0DF0D5
:10146000000EF86E1D0EF76E580EF66E03EC0EF0C1
:1014700088EF02F0F0EC0DF0000EF86E1D0EF76E26
:10148000A80EF66E03EC0EF0200EF2EC0DF07AC111
:101490002CF07BC12DF07CC12EF07DC12FF07EC1E0
:1014A00030F0AFEC16F056EC1AF0080E366E070E60
:1014B000376E3984F8EC19F049EC19F01200F0ECB1
:1014C0000DF0000EF86E1D0EF76EB40EF66E03EC06
:1014D0000EF0200EF2EC0DF07FC12CF080C12DF04B
:1014E00081C12EF082C12FF083C130F056EC1AF08A
:1014F000080E366E060E376E3984F8EC19F049EC9A
:1015000019F012007FC12CF080C12DF081C12EF0A6
:1015100082C12FF083C130F07AC131F07BC132F04B
:101520007CC133F07DC134F07EC135F06CEC14F039
:10153000307E7CEC11F00DC066F10EC067F17FC10A
:101540002CF080C12DF081C12EF082C12FF083C11B
:1015500030F01E0E176E57EC12F0E1EC13F0AFEC0A
:1015600014F07AC131F07BC132F07CC133F07DC11F
:1015700034F07EC135F06CEC14F0307E7CEC11F070
:101580000DC06BF10EC06CF11200F0EC0DF0000E0E
:10159000F86E1D0EF76EEC0EF66E03EC0EF0EAEC34
:1015A0000FF0000EF86E1E0EF76E040EF66E03ECD2
:1015B0000EF066C117F067C118F03EEC1AF0050E88
:1015C000366E1DEC19F0EAEC0FF0000EF86E1E0EF0
:1015D000F76E0C0EF66E03EC0EF06BC117F06CC1DB
:1015E00018F03EEC1AF0050E366E1DEC19F01200E4
:1015F000F0EC0DF0000EF86E1D0EF76EC00EF66EDC
:1016000003EC0EF0200EF2EC0DF07AC117F07BC166
:1016100018F07CC119F07DC11AF07EC11BF00FD803
:10162000400EF2EC0DF07FC117F080C118F081C1BF
:1016300019F082C11AF083C11BF001D812001B50AF
:10164000FAEC0DF01A50FAEC0DF01950FAEC0DF01E
:101650001850FAEC0DF01750FAEC0DF01200706B08
:10166000716B0F0E6F6167D06F6703D0010E706FE3
:101670007CD0010E6F6303D0050E706F76D0020E22
:101680006F6303D00A0E706F70D0030E6F6303D0C8
:101690001E0E706F6AD0040E6F6303D0320E706F2F
:1016A00064D0050E6F6303D0640E706F5ED0060EBB
:1016B0006F6303D0960E706F58D0070E6F6303D020
:1016C000C80E706F52D0080E6F6305D02C0E706F6D
:1016D000010E716F4AD0090E6F6305D0900E706FC6
:1016E000010E716F42D00A0E6F6305D0F40E706F59
:1016F000010E716F3AD00B0E6F6305D0580E706FEC
:10170000020E716F32D00C0E6F6305D0BC0E706F7D
:10171000020E716F2AD00D0E6F6305D0200E706F10
:10172000030E716F22D00E0E6F6305D0840E706FA2
:10173000030E716F1AD0DCEC0FF06FC017F00F0EB4
:101740001C6E5AEC13F0F1EC0FF0C80E1C6EDEECC0
:1017500017F0F1EC0FF0E80E1C6E030E1D6E6FEC2F
:1017600013F017C070F018C071F01200DCEC0FF02D
:10177000440E176E6FC01CF06FEC13F017C006F02C
:101780001200F4DF010E496E20EE58F02BEF0DF041
:10179000EDDF010E496E20EE58F023EC0DF0F1EF75
:1017A0000CF0010E496E20EE6EF00F0E066E23EC6B
:1017B0000DF0F1EF0CF0010E496E20EE6EF00F0E01
:1017C000066E2BEF0DF0DCEC0FF0050E176E6EC001
:1017D0001CF0DEEC17F0100E1C6E6FEC13F017C04F
:1017E00006F01200F0DF050E496E21EE89F023ECC1
:1017F0000DF0F1EF0CF0E7DF050E496E21EE89F0F8
:101800002BEF0DF00A0E496E21EE7AF0040E066EF3
:1018100023EC0DF0F1EF0CF00A0E496E21EE7AF098
:10182000040E066E2BEF0DF0010E496E20EE50F007
:101830000E0E066E23EC0DF0F1EF0CF0010E496E6A
:1018400020EE50F00E0E066E2BEF0DF0010E496EDD
:1018500020EE40F0000E066E23EC0DF0F1EF0CF0E0
:10186000010E496E20EE40F0000E066E2BEF0DF0DB
:10187000010E496E20EE6CF0030E066E23EC0DF0A7
:10188000F1EF0CF0010E496E20EE6CF0030E066EC7
:101890002BEF0DF0010E496E20EE57F0010E066E93
:1018A00023EC0DF0F1EF0CF0010E496E20EE57F035
:1018B000010E066E2BEF0DF0010E496E20EE58F072
:1018C000020E066E23EC0DF0F1EF0CF0010E496EE6
:1018D00020EE58F0020E066E2BEF0DF0010E496E51
:1018E00020EE6FF0420E066E23EC0DF0F1EF0CF0DF
:1018F000010E496E20EE6FF0420E066E2BEF0DF0DA
:10190000F2A400D09EA015D09E90EC0ECF6E780E63
:10191000CE6E526652065366530656665606556696
:1019200008D0545206E054065428D8B45506D8B40A
:1019300054521100006ED8CF01F0E0CF02F002C087
:10194000E0FF005001C0D8FF10000F01700ED36EF1
:10195000806A896A010E926E000E776E816A8A6AC9
:10196000700E936EF00E786E826A8B6A000E946E23
:10197000000ED56EC00EF26E000EF16E000EF06E0F
:10198000000E9D6E000EA06E000E9F6E000EA26EE9
:10199000000ED06E000EC16EBF0EC06E010E7E6EC8
:1019A000000E7F6EEC0ECF6E780ECE6EB50ECD6E45
:1019B0009D800001496800EE00F0EE6A492EFDD7D7
:1019C0001200E5EC0CF0E7EC0CF0E7EC0CF0EDECC1
:1019D0000CF0EDEC0CF0EDEC0CF0FA0E09D0C80EAA
:1019E00007D0640E05D0320E03D00A0E01D0010ECE
:1019F000486E2D0E466E060E476E462EFED7472EBB
:101A0000FCD7482EF6D71200A6B2FED70650A96E14
:101A100005C0A8FFA69EA69CA684F29EF2BEFDD796
:101A2000550EA76EAA0EA76EA68251A4F28EA6949A
:101A30001200A6B2FED70650A96EA69EA69CA6804E
:101A4000A8CF05F01200DECF05F004EC0DF0062A59
:101A5000492EF9D7120019EC0DF005C0DEFF062A59
:101A6000492EF9D71200110E07D00D0E05D0090E20
:101A700003D0050E01D0010EC26EC282C2B2FED7E3
:101A8000C4CF5AF0C3CF59F01200F1EC0CF08B82A6
:101A90008994F1EC0CF08984F1EC0CF08B90F1EC72
:101AA0000CF03A0ED3EC0DF0090ED3EC0DF050B063
:101AB00004D0060ED3EC0DF003D0050ED3EC0DF0E0
:101AC0001E0ED3EC0DF0390ED3EC0DF01B0ED3EC43
:101AD0000DF06E0ED3EC0DF040500F0B700963D873
:101AE0004050E838030B54095ED8380ED3EC0DF0A3
:101AF0000E0ED3EC0DF03A0ED3EC0DF01F0ED3EC1E
:101B00000DF03C0ED3EC0DF06BD81200000EF86E09
:101B10001F0EF76E380EF66E03EC0EF0000EF86E28
:101B20001F0EF76E440EF66E03EC0EF0000EF86E0C
:101B30001F0EF76E500EF66E03EC0EF0E5EC0CF097
:101B4000000EF86E1F0EF76E5C0EF66E03EC0EF0D4
:101B5000000EF86E1F0EF76E680EF66E03EC0EF0B8
:101B6000E5EC0CF0F0EC0DF012003C0ED3EC0DF0B7
:101B70000E0ED3EC0DF012003C0ED3EC0DF00C0E5B
:101B8000D3EC0DF012003D0ED3EC0DF040500F0BD6
:101B9000700909D84050E838030B540904D83C0EAA
:101BA000D3EC0DF012008B90076E1F0E03D08B90BC
:101BB000076E5F0E08D807500F0B05D807380F0BBC
:101BC00002D88B8012003C6E080E3D6E8B923C3228
:101BD000D8A08B94D8B08B848B823D2EF7D712007F
:101BE000010EE1D750A004D03F6E0A0E3F263F50B1
:101BF0008009D9D7086E08380EEC00F0D8DF0850FD
:101C00000EEC00F0D4D70900F550ECDF0900F550D8
:101C100002E0CDDFFBD71200200EC9D73E6E0CECE0
:101C20000EF03E2EFCD71200B5EC0DF0416604D04C
:101C3000290E50A4470E11D0010E416204D0280E87
:101C400050A4450E0AD0020E416202D0420E05D0C9
:101C5000030E416202D0410E00D0F2EC0DF01200F2
:101C6000404133307C2B332C35644200003D3D2015
:101C70005345545550203D00002D2D416262727530
:101C800063682D000064426D2C572C415454200091
:101C900000572C64426D2C41545420000064426D66
:101CA0002C572C4144432000004B616C69627269DF
:101CB00065722E0000566965772D4D6573736B0054
:101CC000004B616C69622E6D616E2E000064426D86
:101CD0002C20646967697400004672714964782039
:101CE00041757300004672714964782045696E0041
:101CF0000046726571752E47616E6700004C434463
:101D0000204B6F6E74722E00004C43442D4472655C
:101D100068656E00202D2D2D2D566F722D2D2D00F6
:101D2000202D2D2D2D4F4B2D2D2D2D00402D2D41B6
:101D30006262727563682D00402D2D5A757275654B
:101D4000636B2D000050313A000000414443313AAA
:101D500000000050323A000000414443323A000093
:101D60002020202B203164426D2020004020202D97
:101D7000203164426D202000004162627275636808
:101D80002121210000576965646572682E212100B8
:101D9000002D2D5765697465722D2D0000537065F7
:101DA00069636865726E2100004D6B78202A2031CE
:101DB00030303000004D6B79202020202020200082
:101DC000004D6B787920202048455800004B6F6EFD
:101DD00074723A00202B204B6F6E74726173740022
:101DE000402D204B6F6E7472617374000041444348
:101DF0002D57657274652000002D2D4B7572736F21
:101E0000722D2D0020414443313A000040414443AB
:101E1000323A0000005461737465204C616E6700B3
:101E2000202D46756E6B74696F6E2D00002D2D2070
:101E300053617665202D2D00202D416262727563FD
:101E4000682D2D00402D416262727563682D2D0052
:101E5000402D2D5765697465722D2D00003D64423B
:101E60006D204D61783D3D00202D5370656963689C
:101E700065722D00402D2D6C6573656E2D2D2D0026
:101E8000202D2D2D2D434C522D2D2D00202D537006
:101E90006569636865726E00402D4265656E6465B4
:101EA0006E2D2D000053702E506C61747A3A000034
:101EB000205370656963686572202B00405370651C
:101EC0006963686572202D000064426D2044696773
:101ED00069742000204469676974203D2033200024
:101EE000404469676974203D20342000404F666695
:101EF0000000082D5600082D4500002D20436C6F72
:101F00007365202D2D00002D204C65747A74657248
:101F10002D00202D204F6666736574202D00402D06
:101F200020644220576572742D00503D00004144EA
:101F3000433D00004D487A00003D6D572D4D6574BE
:101F400065723D00204857312E303120202020007E
:101F5000405357312E303420202020002032342EA0
:101F600030342E323032300040286329444C344A19
:101F7000414C20002D2D2D00494E46006D5700008C
:101F8000755700006E57000070570000665700003C
:101F900061570000572000006B57000020560000DA
:101FA0006D560000755600006E56000064426D00CC
:101FB000644200007373000013D806D8126A136AD3
:101FC000146A156A166A12000D6A0E6A0F6A106AA0
:101FD000116A1200176A186A196A1A6A1B6A1200D3
:101FE000F9DF1C6A1D6A1E6A1F6A206A12002C6AC9
:101FF0002D6A2E6A2F6A306A12000EC131F00FC1AD
:1020000032F010C133F011C134F012C135F01200BA
:102010000EC12CF00FC12DF010C12EF011C12FF008
:1020200012C130F0120031C02CF032C02DF033C09C
:102030002EF034C02FF035C030F012002CC031F03B
:102040002DC032F02EC033F02FC034F030C035F048
:1020500012002CC00EF12DC00FF12EC010F12FC0B8
:1020600011F130C012F1120013C12CF014C12DF087
:1020700015C12EF016C12FF017C130F0120013C198
:1020800031F014C132F015C133F016C134F017C16C
:1020900035F0120018C12CF019C12DF01AC12EF024
:1020A0001BC12FF01CC130F0120018C131F019C152
:1020B00032F01AC133F01BC134F01CC135F01200EC
:1020C0001DC12CF01EC12DF01FC12EF020C12FF01C
:1020D00021C130F012001DC131F01EC132F01FC10C
:1020E00033F020C134F021C135F0120022C12CF0B0
:1020F00023C12DF024C12EF025C12FF026C130F0D0
:10210000120022C131F023C132F024C133F025C1C5
:1021100034F026C135F0120027C12CF028C12DF073
:1021200029C12EF02AC12FF02BC130F0120027C197
:1021300031F028C132F029C133F02AC134F02BC16B
:1021400035F0120031C013F132C014F133C015F173
:1021500034C016F135C017F112002CC013F12DC098
:1021600014F12EC015F12FC016F130C017F1120076
:102170002CC018F12DC019F12EC01AF12FC01BF17F
:1021800030C01CF112002CC01DF12DC01EF12EC05C
:102190001FF12FC020F130C021F112002CC022F11C
:1021A0002DC023F12EC024F12FC025F130C026F11F
:1021B00012002CC027F12DC028F12EC029F12FC00C
:1021C0002AF130C02BF112000DC017F00EC018F02C
:1021D0000FC019F010C01AF011C01BF012000DC092
:1021E0001CF00EC01DF00FC01EF010C01FF011C07B
:1021F00020F0120017C00DF018C00EF019C00FF03B
:102200001AC010F01BC011F012001C361D361E360D
:102210001F36203612001736183619361A361B3676
:10222000120020321F321E321D321C3212001B32AD
:102230001A32193218321732120006D812361336F3
:1022400014361536163612000D360E360F36103689
:1022500011361200163215321432133212321200B5
:10226000F9DF113210320F320E320D32120017AE7A
:1022700004D0186819681A681B68120018AE03D0D9
:1022800019681A681B68120019AE02D01A681B6818
:1022900012001AAE01D01B6812003A9239BE3A827F
:1022A0008CDE280E0A6ED89017EC11F031EC11F08C
:1022B00003D80A2EF8D7120020EC1BF00A0E096E84
:1022C00000EE0DF0EF50E8B6FD0FE8BED00FEE6E59
:1022D000092EF8D72DEC1BF012003FD811AE09D013
:1022E000122AD8B4132AD8B4142AD8B4152AD8B4C8
:1022F000162AE4EC0FF035D030D811AE09D0122AEE
:10230000D8B4132AD8B4142AD8B4152AD8B4162AA3
:1023100012C00DF013C00EF014C00FF015C010F075
:1023200016C011F039BE25EC18F0120016D812C0F4
:102330000DF013C00EF014C00FF015C010F016C051
:1023400011F039BE25EC18F0120007D8DEEC0FF0C2
:1023500008D003D8E4EC0FF004D0C0EC13F0B5EFD4
:1023600011F072EC12F0D6EF13F04CD803E1DDEC73
:102370000FF01AD01AD87F0E216E2150255E225000
:10238000265A25C009F025520FE025BE06D0D89068
:102390001DEC11F0092EFBD707D0091E092AD89091
:1023A00030EC11F0092EFBD71200399E2BBE398E6E
:1023B0002B9EDDEC0FF027C00EF028C00FF029C0D7
:1023C00010F02AC011F02BC012F0D8901DEC11F0C3
:1023D00031EC11F0118E12C025F0126AD8901DEC6C
:1023E00011F01200040E096EEE6608D0092EFCD71B
:1023F000EECFE8FF7F0B03E1D88401D0D8942DEC19
:102400001BF0120020EC1BF000EE27F0EBD720ECC5
:102410001BF000EE2CF0E6D720EC1BF000EE31F0C4
:10242000E1D720EC1BF000EE17F0DCD720EC1BF01E
:1024300000EE1CF0D7D720EC1BF000EE0DF00A0EDA
:10244000096EEE66DBD7092EFCD7D6D71B6A1ABEFB
:102450001B6835D01A6A1B6A19AE31D01A681B681E
:102460002ED0196A1A6A1B6A18AE29D019681A6820
:102470001B6825D0186A196A1A6A1B6A17AE1FD022
:10248000186819681A681B681AD0DDEC0FF0399EBD
:102490001B6A1DD0DDEC0FF0399E1A6A1B6A17D03B
:1024A000DDEC0FF0399E196A1A6A1B6A10D0DDEC58
:1024B0000FF0399E186A196A1A6A1B6A08D0DDEC97
:1024C0000FF0399E1BAE03D034EC18F0398E17C0D4
:1024D00012F018C013F019C014F01AC015F01BC088
:1024E00016F000D07F0E256E000E266E1BEC12F04B
:1024F00006E1276A286A296A2A6A2B6A36D0DCEC48
:1025000012F007E0D89030EC11F0252AD8B4262A32
:10251000F6D712B00AD0D8901DEC11F02506252868
:10252000D8B42606D8B42552F4D70EA00BD00E800E
:102530000E2AD8B40F2AD8B4102AD8B4112AD8B485
:10254000122ADDD70D6A129025C012F030EC11F07E
:102550000EC027F00FC028F010C029F011C02AF0DB
:1025600012C02BF02B9E39BE2B8E1200276A286AD0
:10257000296A2B6A800E2A6EF5D727682868296891
:102580007F0E2A6E7F0E2B6EEDD77F0E176E000E1C
:10259000186E2650185C02E12550175CD8B003D0A5
:1025A000ECDFD88401D0D894120026AE03D0DEDF51
:1025B000D88401D0D894120020EC1BF000EE16F065
:1025C000040E096EED660AD0092EFCD7010EEF62EB
:1025D00001D002D0EF6602D0D88401D0D8942DEC7F
:1025E0001BF012001CC000F11DC001F11EC002F161
:1025F0001FC003F120C004F13CEC13F00DC007F143
:102600000EC008F10FC009F110C00AF111C00BF1A2
:1026100000C117F001C118F002C119F003C11AF08E
:1026200004C11BF022EC13F007C112F008C113F033
:1026300009C114F00AC115F00BC116F0399E3AB267
:10264000398E1200BADC280E0A6ED89005D824EC18
:1026500011F00A2EFAD7120020EC1BF0050E096EBD
:1026600000EE17F0D890EF50E8200700EE6E092E2C
:10267000FAD72DEC1BF0120020EC1BF09EDC280E8C
:102680000A6ED89017EC11F031EC11F000EE17F053
:10269000050E096EEFAE02D0300EEF5EEFA602D04F
:1026A000030EEF5EEE52092EF5D70A2EEAD72DEC77
:1026B0001BF0120002D8E4EF10F020EC1BF09ADDC2
:1026C00000EE0DF010EE1CF0040E096EE650EE5E0A
:1026D000E650EE5A092EFCD72DEC1BF0120002D862
:1026E000E4EF10F020EC1BF085DD00EE0DF010EEB5
:1026F0001CF0E650EE26040E096EE650EE22092E7E
:10270000FCD72DEC1BF0120000C117F001C118F02E
:1027100002C119F003C11AF004C11BF005C121F078
:1027200006C122F0120007C11CF008C11DF009C14A
:102730001EF00AC11FF00BC120F00CC123F00DC127
:1027400024F012000EC000F10FC001F110C002F120
:1027500011C003F112C004F125C005F126C006F135
:1027600012000EC007F10FC008F110C009F111C02E
:102770000AF112C00BF125C00CF126C00DF11200B8
:102780002CC027F02DC028F02EC029F02FC02AF031
:1027900030C02BF0120031C027F032C028F033C017
:1027A00029F034C02AF035C02BF0120027C02CF0DD
:1027B00028C02DF029C02EF02AC02FF02BC030F0F9
:1027C000120027C031F028C032F029C033F02AC0EF
:1027D00034F02BC035F012003DEC1BF016E23AEC61
:1027E0001BF013E207EC12F01AE00CEC12F017E009
:1027F00052EC1BF004E307EC12F001E306D055ECB9
:102800001BF006E30CEC12F003E37AEC1BF0120071
:1028100052EC1BF003E36FEC1BF003D00DD0F7EC90
:102820000FF030BE03D035AE01D0308E30AE03D0C5
:1028300035BE01D0308E12001DD8399E39BA397E8E
:1028400039BC397EE1EC17F011C000F112C001F182
:1028500013C002F114C003F115C004F11ED872ECCC
:1028600013F0E4EC10F0F1EC0FF07F0E1C6E5DEC59
:1028700013F01ED0399A399C30BE398A35BE398C56
:102880007FDFD5EC11F05EDF86DFD5EC11F069DF7C
:10289000DCEC0FF039DF93EF13F0DCEC0FF021C02C
:1028A00017F022C018F023C01CF024C01DF0120045
:1028B0000DC025F00EC026F0DDEC0FF000C10EF0CB
:1028C00001C10FF002C110F003C111F004C112F0F8
:1028D00076EC12F0D6EF13F03DEC1BF009E23AEC87
:1028E0001BF006E207EC12F006E10CEC12F019E125
:1028F0007AEC1BF0120055EC1BF003E352EC1BF0DA
:10290000F7E20CEC12F010E16FEC1BF030BE03D0DC
:1029100035AE01D0308E30AE03D035BE01D0308E12
:10292000120084EC1BF0F2D7A5DF399E39BA397E4C
:1029300039BC397EAFEC18F005DFAFDF5DEC13F08A
:10294000E4EC10F0F1EC0FF07F0E1C6E72EC13F063
:10295000AFD70CEC12F001E11200357E00D03DEC57
:102960001BF004E23AEC1BF001E203D07AEC1BF01E
:1029700012000CEC12F001E1120007EC12F003E17E
:1029800013EC10F0120017D872EC13F021C025F0F0
:1029900022C026F0399E11AE03D0398E25EC18F0F6
:1029A0000DC000F10EC001F10FC002F110C003F123
:1029B00011C004F181D75EDFFE0E256E000E266E7B
:1029C0002450225C02E12350215C27E013E3232AF8
:1029D000D8B4242A2650245C02E12550235C07E168
:1029E000F1EC0FF021C023F022C024F016D0D890D3
:1029F00018DCE6D7212AD8B4222A2650225C02E12C
:102A00002550215C07E1EAEC0FF023C021F024C03F
:102A100022F003D0D8900BDCD3D739BA34EC18F0BD
:102A200039BC43EC18F012001EEC10F0ECEF13F080
:102A300007EC12F02DE030BE2CD03DEC1BF028E26C
:102A400029EC10F0ECD848DFADEC10F01E0E0C6E47
:102A50000C4E1ED008EC10F03FEC10F03DDF3FECC8
:102A600010F07DDFDCD838DF3FEC10F03550305C03
:102A70000BE134502F5C08E133502E5C05E13250FD
:102A80002D5C02E131502C5C03E0ADEC10F0E0D79E
:102A900012007AEC1BF0120007EC12F008E13F0E76
:102AA000306E800E2F6E2C6A2D6A2E6A1200010184
:102AB0003F0E266F800E256F226B236B246B3F0E1B
:102AC000216F800E206F1D6B1E6B1F6B0001B8EC19
:102AD00010F0ADEC10F022C10EF123C10FF124C1B2
:102AE00010F125C111F126C112F11E0E0C6E34EC4D
:102AF00010F06BEC10F0F0DEFDEC0FF0AFEC14F02A
:102B0000FDEC0FF03550305C0BE134502F5C08E1E8
:102B100033502E5C05E132502D5C02E131502C5CCB
:102B200017E00C4E15D029EC10F076EC10F06FD8B1
:102B300016DFCEEC10F06BEC10F04EDEC3EC10F0B4
:102B40004AEC10F03FEC10F047DEADEC10F0CFD7C0
:102B5000120007EC12F008E13F0E306E800E2F6E6F
:102B60002C6A2D6A2E6A12002CC02CF12DC02DF17A
:102B70002EC02EF12FC02FF130C030F1A5EC11F096
:102B80003BD82ADE89DFD9EC10F02CC12CF02DC106
:102B90002DF02EC12EF02FC12FF030C130F0ADEC52
:102BA00011F0399439BE398412C00CF027C12CF0D1
:102BB00028C12DF029C12EF02AC12FF02BC130F0F1
:102BC0000C5206E039A4C5D839B4D5D80C2EFAD7A2
:102BD0001200420E356E480E346E316A326A336A24
:102BE0001200400E356E490E346E0F0E336EDA0E43
:102BF000326EA20E316E1200400E356E130E346E20
:102C00005D0E336E8D0E326EDE0E316E12003F0E93
:102C1000356E800E346E316A326A336A1200400EAD
:102C2000356E316A326A336A346A1200410E356E8B
:102C3000200E346E316A326A336A1200420E356EEB
:102C4000C80E346E316A326A336A1200440E356E31
:102C50007A0E346E316A326A336A1200460E356E6D
:102C60001C0E346E400E336E316A326A1200470E0B
:102C7000356EC30E346E500E336E316A326A1200F6
:102C8000490E356E740E346E240E336E316A326A1C
:102C900012004B0E356E180E346E960E336E800E8B
:102CA000326E316A12004C0E356EBE0E346EBC0EA2
:102CB000336E200E326E316A12004E0E356E6E0E7D
:102CC000346E6B0E336E280E326E316A12003D0E7A
:102CD000356ECC0E346ECC0E336ECC0E326ECD0E05
:102CE000316E12003C0E356E230E346ED70E336EED
:102CF0000A0E326E3D0E316E12003A0E356E830EA4
:102D0000346E120E336E6E0E326E980E316E1200ED
:102D1000350E356E860E346E370E336EBD0E326E46
:102D2000060E316E1200300E356E890E346E700E46
:102D3000336E5F0E326E410E316E12002B0E356E09
:102D40008C0E346EBC0E336ECC0E326E090E316EAC
:102D500012006CDFECEF13F071DFECEF13F076DFB5
:102D6000ECEF13F07BDFECEF13F081DFECEF13F00F
:102D700087DFECEF13F05ADF6CEF14F05FDF6CEFDE
:102D800014F064DF6CEF14F069DF6CEF14F06FDFA8
:102D90006CEF14F075DF6CEF14F007EC12F003E148
:102DA0007AEC1BF0120029EC10F001013F0E176FB6
:102DB000800E166F136B146B156B000128DFA9ECE6
:102DC00014F0B8EC10F008EC10F021DFAFEC14F0C8
:102DD000C3EC10F04AEC10F06BEC10F06CEC14F05B
:102DE000B8EC10F0CEEC10F029EC10F0280E0C6EC0
:102DF00034EC10F014DFAFEC14F0ADEC10F04AEC52
:102E000010F081EC10F0ECEC13F081EC10F0ECEC35
:102E100013F0B8EC10F03FEC10F06CEC14F0FDEC9B
:102E20000FF0AFEC14F0FDEC0FF03550305C0BE11F
:102E300034502F5C08E133502E5C05E132502D5C9C
:102E400002E131502C5C05E00C4E03D029EC10F06F
:102E5000CFD7E5DEECEF13F00101276B000116EC94
:102E600016F048D806E3BBEC16F00101272B000151
:102E7000F6D793DFC1DE6CEC14F0DCEC0FF027C169
:102E800012F0125206E072EC12F0E1EC13F0AFEC2B
:102E900014F012007ED81BAE14D020AE29D05AD820
:102EA0001B50205C0BE11A501F5C08E119501E5C9E
:102EB00005E118501D5C02E117501C5CD8B016D01B
:102EC00017D01BBE02D020BE11D044D81B50205CAE
:102ED0000BE11A501F5C08E119501E5C05E1185007
:102EE0001D5C02E117501C5CD8B002D0D89001D014
:102EF000D88012004ED81BAE14D020AE29D02AD8CC
:102F00001B50205C0BE11A501F5C08E119501E5C3D
:102F100005E118501D5C02E117501C5CD8B016D0BA
:102F200017D01BBE02D020BE11D014D81B50205C7D
:102F30000BE11A501F5C08E119501E5C05E11850A6
:102F40001D5C02E117501C5CD8B002D0D88001D0C3
:102F5000D890120007EC12F003E1EAEC0FF00FD06A
:102F6000D8900BEC11F0D8901A321932183217326F
:102F70001A8E0CEC12F003E1F1EC0FF009D0D890AE
:102F800005EC11F0D8901F321E321D321C321F8EFC
:102F900012002CC017F02DC018F02EC019F02FC051
:102FA0001AF030C01BF031C01CF032C01DF033C02D
:102FB0001EF034C01FF035C020F0120002D8E4EF3C
:102FC00010F020EC1BF037D8050E096E00EE1CF057
:102FD00020EE0DF0DDEC0FF010EE17F0050E0A6E8E
:102FE00009C00BF00A500B260B060B06EF50E60249
:102FF000F350DE26D9CF36F0DACF37F0F450DE22A8
:10300000E86ADE220B2EFCD736C0D9FF37C0DAFFC4
:103010000A2EE6D7EE5220EE0DF0060E0B6E09508A
:103020000B5EDE520B2EFDD7092ED6D72DEC1BF0F2
:1030300039B20BD8120039921BAE02D015D83972B2
:1030400020AE02D020D8397212000D1E0E1E0F1EA7
:10305000101E111E0D2AD8B40E2AD8B40F2AD8B4C7
:10306000102AD8B4112A1200171E181E191E1A1E73
:103070001B1E172AD8B4182AD8B4192AD8B41A2A69
:10308000D8B41B2A12001C1E1D1E1E1E1F1E201E31
:103090001C2AD8B41D2AD8B41E2AD8B41F2AD8B4E2
:1030A000202A1200C8DF20EC1BF0DDEC0FF0050E2B
:1030B000096E00EE1CF0EE6605D0092EFCD72DEC53
:1030C0001BF01200096A092AD89020BE1CD01C36B9
:1030D0001D361E361F36203620501B5C0BE11F505C
:1030E0001A5C08E11E50195C05E11D50185C02E1F4
:1030F0001C50175CE8E2DDEC0FF0D89020321F3254
:103100001E321D321C3220501B5C0BE11F501A5C1A
:1031100008E11E50195C05E11D50185C02E11C50CD
:10312000175C0AE31C50175E1D50185A1E50195A9E
:103130001F501A5A20501B5A24EC11F0092EDDD7CB
:1031400077DF17C01CF018C01DF019C01EF01AC0A0
:103150001FF01BC020F0E4EC10F02DEF1BF0290E47
:10316000096EDDEC0FF020501B5C0BE11F501A5C68
:1031700008E11E50195C05E11D50185C02E11C506D
:10318000175C0BE31C50175E1D50185A1E50195A3D
:103190001F501A5A20501B5AD8801DEC11F0D8909D
:1031A0000BEC11F020501B5C0BE11F501A5C08E186
:1031B0001E50195C05E11D50185C02E11C50175CA3
:1031C0000BE31C50175E1D50185A1E50195A1F5001
:1031D0001A5A20501B5AD880092EDFD7120020EC33
:1031E0001BF039921BAE02D03FDF3982DDEC0FF0CD
:1031F000280E096E0A0E0A6E00EE0DF0EF500F0B4E
:103200000B6E050E0B5CD8A002D0030EEF26EF501C
:10321000F00B0B6E500E0B5CD8A002D0300EEF26D8
:10322000EC520A2EEBD7D8900BEC11F01DEC11F0FC
:10323000092EE0D72DEC1BF012003DEC1BF015E23F
:1032400055EC1BF01CE22FD844D85AD83A941200FF
:10325000030E366409D03766362A39B4362A030E8F
:10326000365E36500EEC0EF01200F2DF000EF86EF5
:103270001F0EF76E740EF66E06EC0EF01200E8DF0D
:10328000000EF86E1F0EF76E780EF66E06EC0EF05E
:1032900012003DEC1BF0E9E255EC1BF0F0E203D824
:1032A0002FD83A94120020EC1BF000EE16F011EE2D
:1032B00031F00A0E0B6EEDCF09F009380A6E56D8C0
:1032C00009C00AF053D80B2EF6D7E76A2DEC1BF095
:1032D000120020EC1BF0375210E001EE44F011EE2A
:1032E00044F0140E096E37C00AF0E55009060A2EA4
:1032F000FCD7E5CFEDFF092EFCD72DEC1BF012001B
:1033000020EC1BF00A0E0A6E37500A2636500A5C73
:10331000D8B002D00AC036F03650375CD8A003D0FF
:1033200037C036F0362A3750365E3606090E096E3B
:103330003650095E01EE31F0095204E0EECFE8FFAD
:10334000092EFCD739A405D02B0E39BE2D0EF5EC75
:1033500019F0398019D8399013D8375204E02C0E5F
:10336000F5EC19F009D82DEC1BF012000A500F0BE8
:103370003009E8CFE6FF120037C00BF03A9606D0CE
:10338000010E0B6E3A9602D036C00BF00B5226E0BF
:1033900039A006D0EFCF09F0300E095CD8A43990DF
:1033A0003AA611D00BC017F0020E176202D0EFEC54
:1033B00019F0050E176202D0EFEC19F0080E176233
:1033C00002D0EFEC19F0EECFE8FF39B003D0F5EC06
:1033D00019F002D0F1EC19F00B2EDAD71200200E02
:1033E00004D0200E3AB4300E00D0D7EC0DF012000D
:1033F00020EC1BF00A0E096E3750095E00EE0DF04E
:10340000EF50094E0CD0EF50094E02D0EE52F8D7D3
:10341000EE52176E490E176409D0010E06D00F0B3D
:10342000176E040E176402D0100EEF260A0E096EF6
:1034300000EE0DF0EF500700EE6EE86AEF22092E65
:10344000F9D72DEC1BF0120020EC1BF0050E096ED5
:103450000A0E0A6E00EE16F0EDCF17F01750F00BC3
:1034600007E10A0617500F0B03E10A06092EF4D7ED
:103470000AC017F00A502DEC1BF0120084EC1BF070
:10348000DDEC0FF0EFEC18F00DC012F00EC013F0F1
:103490000FC014F010C015F011C016F0050E366EF6
:1034A000376A39943A9439983A9612003DEC1BF0F9
:1034B00044E255EC1BF041E2C0EC13F0B5EC11F026
:1034C0000DC000F10EC001F10FC002F110C003F1F8
:1034D00011C004F112C017F013C018F014C019F095
:1034E00015C01AF016C01BF0EFEC18F00DC007F174
:1034F0000EC008F10FC009F110C00AF111C00BF1A4
:1035000000C117F001C118F002C119F003C11AF08F
:1035100004C11BF04DEC11F007C112F008C113F00B
:1035200009C114F00AC115F00BC116F0140E366E65
:103530000A0E376E39983A963A943994120029EC6B
:1035400010F0386A309E07EC12F014E016EC16F01A
:103550007AEC17F001E004E3BBEC16F0382AF6D75A
:1035600007EC16F04AEC17F005E004E3A9EC16F0BE
:103570003806F6D756EC1AF008EC10F030BE398E4B
:103580000B0E366E0A0E376E39843998120049ECEC
:1035900019F0650EF5EC19F0399E38BE398E38BE3B
:1035A000386CEAEC0FF038C017F03EEC1AF03984B2
:1035B0004BDF17C036F049EC19F0120034EC10F074
:1035C000FDEC0FF0A9EC14F0D9EC10F060EC10F069
:1035D00055EC10F0A9EC14F01EEC10F027C12CF003
:1035E00028C12DF029C12EF02AC12FF02BC130F0B7
:1035F0006CEC14F0D9EC10F076EC10F055EC10F007
:10360000A9EC14F097EC10F0ECEC13F0FDEC0FF0DB
:10361000AFEC14F0120020EC1BF0EAEC0FF0050EFA
:10362000096E10EE0DF020EE17F0E6500F0BDF6E76
:10363000E638F00BDE12092EF8D72DEC1BF0120045
:10364000E9CF45F1EACF46F1E1CF47F1E2CF48F1CA
:10365000D9CF49F1DACF4AF1120045C1E9FF46C19D
:10366000EAFF47C1E1FF48C1E2FF49C1D9FF4AC1B2
:10367000DAFF1200CBEC13F003D0C0EC13F000D053
:103680002B9E7F0E2B620CD0800E2A6207D02966FB
:1036900005D0286603D0276601D002D0D88001D09B
:1036A000D8901200CBEC13F003D0C0EC13F000D094
:1036B0002B9E7F0E2B620BD0800E2A6208D02966CB
:1036C00006D0286604D0276602D0D88001D0D890D2
:1036D000120002D8D6EF13F005D82B8E120002D8B4
:1036E000D6EF13F07F0E2B6E800E2A6E276A286AA3
:1036F000296A120002D8D6EF13F07F0E2B6E2768CE
:10370000286829682A68120002D8D6EF13F0276AC1
:10371000286A296A2A6A2B6A1200410E356EA00EA9
:10372000346E316A326A336A12008DEC1BF06CEC35
:1037300014F0A9EC15F029EC10F007EC16F0AFEC42
:1037400014F0ADEC10F008EC10F007EC16F0A9EC5A
:1037500014F01EEC10F034EC10F06CEC14F01200CD
:103760004BC12CF04CC12DF04DC12EF04EC12FF0AD
:103770004FC130F0BBEC16F0A9EC15F02CC055F1A0
:103780002DC056F12EC057F12FC058F130C059F15D
:10379000120055C12CF056C12DF057C12EF058C162
:1037A0002FF059C130F0C1EC16F0E9EC15F0ECEC5B
:1037B00013F018EC15F02CC060F12DC061F12EC093
:1037C00062F12FC063F130C064F1120060C12CF0CF
:1037D00061C12DF062C12EF063C12FF064C130F0E1
:1037E0000101010E656F000188EC16F04AEC17F03C
:1037F00009E30101040E656F0001B8EC16F0AFECAF
:1038000016F018D07DEC16F04AEC17F007E3010132
:10381000030E656F0001B8EC16F00CD007EC16F043
:103820004AEC17F007E30101020E656F0001AFECEF
:1038300016F000D02CC05BF12DC05CF12EC05DF104
:103840002FC05EF130C05FF1120055C12CF056C19F
:103850002DF057C12EF058C12FF059C130F00101A1
:10386000030E5A6F00019EEC16F04AEC17F00BE3C2
:10387000B8EC16F0B8EC16F0AFEC16F00101080E3B
:103880005A6F00014CD093EC16F04AEC17F009E3A4
:10389000B8EC16F0B8EC16F00101070E5A6F0001F3
:1038A0003ED088EC16F04AEC17F009E3B8EC16F0BD
:1038B000AFEC16F00101060E5A6F000130D07DEC1E
:1038C00016F04AEC17F007E3B8EC16F00101050E0C
:1038D0005A6F000124D007EC16F04AEC17F007E30A
:1038E000AFEC16F00101040E5A6F000118D040EC45
:1038F00016F07AEC17F007E3CAEC16F00101010E9E
:103900005A6F00010CD026EC16F07AEC17F007E3A2
:10391000C1EC16F00101020E5A6F000100D02CC05C
:1039200050F12DC051F12EC052F12FC053F130C0D3
:1039300054F1120050C12CF051C12DF052C12EF0A3
:1039400053C12FF054C130F056EC1AF0050E366E0C
:10395000010E376E16EC16F04AEC17F003E3040E76
:10396000376E0FD01EEC16F04AEC17F003E3030E8F
:10397000376E07D026EC16F04AEC17F002E3020E81
:10398000376E67D8F8EC19F049EC19F05AC117F006
:10399000030E176209D0000EF86E1F0EF76E7C0E34
:1039A000F66E06EC0EF054D0040E176209D0000E2D
:1039B000F86E1F0EF76E800EF66E06EC0EF048D015
:1039C000050E176209D0000EF86E1F0EF76E840EFA
:1039D000F66E06EC0EF03CD0060E176209D0000E13
:1039E000F86E1F0EF76E880EF66E06EC0EF030D0F5
:1039F000070E176209D0000EF86E1F0EF76E8C0EC0
:103A0000F66E06EC0EF024D0020E176209D0000EFE
:103A1000F86E1F0EF76E940EF66E06EC0EF018D0D0
:103A2000010E176209D0000EF86E1F0EF76E980E89
:103A3000F66E06EC0EF00CD0080E176209D0000EE0
:103A4000F86E1F0EF76E900EF66E06EC0EF000D0BC
:103A5000120024EC1AF0030E176402D0010E376E28
:103A6000030E176202D0020E376E020E176202D0EA
:103A7000030E376E010E176202D0040E376E000E71
:103A8000176202D0040E376E12005BC12CF05CC1CD
:103A90002DF05DC12EF05EC12FF05FC130F056EC0D
:103AA0001AF0060E366E010E376E26EC16F04AEC52
:103AB00017F002E3020E376E1EEC16F04AEC17F018
:103AC00002E3030E376E16EC16F04AEC17F002E331
:103AD000040E376EBEDFF8EC19F049EC19F065C141
:103AE00017F0010E176209D0000EF86E1F0EF76E68
:103AF0009C0EF66E06EC0EF024D0020E176209D072
:103B0000000EF86E1F0EF76EA00EF66E06EC0EF0AD
:103B100018D0030E176209D0000EF86E1F0EF76E54
:103B2000A40EF66E06EC0EF00CD0040E176209D04F
:103B3000000EF86E1F0EF76EA80EF66E06EC0EF075
:103B400000D012004BC12CF04CC12DF04DC12EF015
:103B50004EC12FF04FC130F056EC1AF0050E366E04
:103B6000020E376EF8EC19F024EC1AF0030E176011
:103B700004D0040E366E020E376E020E176404D0A7
:103B8000040E366E010E376E24D04BC12CF04CC1A2
:103B90002DF04DC12EF04EC12FF04FC130F056EC3C
:103BA0001AF0040E366E010E376EF8EC19F024ECA4
:103BB0001AF0030E176004D0030E366E010E376E36
:103BC000020E176406D0040E366E000E376EF8EC47
:103BD00019F0398449EC19F0000EF86E1F0EF76EDB
:103BE000AC0EF66E06EC0EF0120050C12CF051C176
:103BF0002DF052C12EF053C12FF054C130F056ECCD
:103C00001AF0040E366E010E376E16EC16F04AEC02
:103C100017F003E3030E376E0FD01EEC16F04AECDC
:103C200017F003E3020E376E07D026EC16F04AECCD
:103C300017F002E3010E376EF8EC19F065D849EC85
:103C400019F05AC117F0030E176209D0000EF86E72
:103C50001F0EF76E7C0EF66E06EC0EF054D0040EBE
:103C6000176209D0000EF86E1F0EF76E800EF66E0A
:103C700006EC0EF048D0050E176209D0000EF86E63
:103C80001F0EF76E840EF66E06EC0EF03CD0060E9C
:103C9000176209D0000EF86E1F0EF76E880EF66ED2
:103CA00006EC0EF030D0070E176209D0000EF86E49
:103CB0001F0EF76E8C0EF66E06EC0EF024D0020E80
:103CC000176209D0000EF86E1F0EF76E940EF66E96
:103CD00006EC0EF018D0010E176209D0000EF86E37
:103CE0001F0EF76E980EF66E06EC0EF00CD0080E56
:103CF000176209D0000EF86E1F0EF76E900EF66E6A
:103D000006EC0EF000D0120024EC1AF0030E17643B
:103D100004D0050E366E000E376E030E176202D009
:103D2000010E376E020E176202D0020E376E010EC0
:103D3000176202D0030E376E000E176202D0030E18
:103D4000376E120050C12CF051C12DF052C12EF02F
:103D500053C12FF054C130F056EC1AF0030E366EFA
:103D6000010E376E16EC16F04AEC17F003E3020E64
:103D7000376E11D01EEC16F04AEC17F003E3010E7B
:103D8000376E09D026EC16F04AEC17F004E3000E6B
:103D9000376E040E366EF8EC19F065D849EC19F060
:103DA0005AC117F0030E176209D0000EF86E1F0EED
:103DB000F76E7C0EF66E06EC0EF054D0040E176211
:103DC00009D0000EF86E1F0EF76E800EF66E06EC30
:103DD0000EF048D0050E176209D0000EF86E1F0EC7
:103DE000F76E840EF66E06EC0EF03CD0060E1762EF
:103DF00009D0000EF86E1F0EF76E880EF66E06ECF8
:103E00000EF030D0070E176209D0000EF86E1F0EAC
:103E1000F76E8C0EF66E06EC0EF024D0020E1762D2
:103E200009D0000EF86E1F0EF76E940EF66E06ECBB
:103E30000EF018D0010E176209D0000EF86E1F0E9A
:103E4000F76E980EF66E06EC0EF00CD0080E1762A8
:103E500009D0000EF86E1F0EF76E900EF66E06EC8F
:103E60000EF000D0120024EC1AF0030E176404D0F8
:103E7000040E366E000E376E030E176204D0040E69
:103E8000366E000E376E020E176202D0010E376ECC
:103E9000010E176202D0020E376E000E176202D0BA
:063EA000020E376E120055
:020000040030CA
:0300010028191E9D
:02000500088071
:0200000400F00A
:100000002D0A00003DE9F082BBAE9873CC4105009B
:1000100000000000000000000000000000000000E0
:1000200000000000000000000000000000000000D0
:1000300000000000000000000000000000000000C0
:100040000000160000000000FFFEFDFAF8F6F5F1D2
:10005000F2EFECEAE9E6DFD9D2CBC5C5CFDBD700BA
:100060000000000000000000000000000000000090
:08007000000000000000000088
:00000001FF
